:020000040000FA
:0600000058EF07F01200AA
:0608000058EF07F01200A2
:06082A000100CE0E0000EB
:0808300000020000200000009E
:08083800D9CFE6FFE1CFD9FFA3
:10084000040EE126DE6ADE6ADE6ADD6ADD52DD5212
:10085000FB0EDBCF00F0FC0EDBCF01F0FD0EDBCF9B
:1008600002F0FE0EDBCF03F0D9CFE9FFDACFEAFFCB
:10087000030EEB500318E8AE02D0033408D000504A
:10088000EE5C0150EE580250EE580350EE580FE265
:100890000C0EE66E38EC07F0E552D9CFE9FFDACF5F
:1008A000EAFFEE2A000EEE22EE22EE22D1D7040E4F
:1008B000E15C02E2E16AE552E16EE552E7CFD9FF81
:1008C00012000F0EC16E070EB46E936A816A300E6D
:1008D000926E0F0E946EF19E1200D9CFE6FFE1CF1B
:1008E000D9FF020EE1268250020B01E0010E080D35
:1008F000F3CF02F08250010B040DF3CF01F08050D2
:10090000200B01E0010EE824006E8050100B01E086
:10091000010E002401240224DE6EDD6ADECF00F029
:10092000DDCF01F000C0F3FF01C0F4FF020EE15C77
:1009300003E200D0E16AE552E16EE552E7CFD9FF6C
:1009400012008092010EE66EE66AE66AE66A74DFDD
:10095000E552E552E552E5528084010EE66EE66A04
:10096000E66AE66A69DFE552E552E552E5528094AF
:10097000010EE66EE66AE66AE66A5EDFE552E55279
:10098000E552E55212008082010EE66EE66AE66AE2
:10099000E66A52DFE552E552E552E5528084010EE7
:1009A000E66EE66AE66AE66A47DFE552E552E55238
:1009B000E5528094010EE66EE66AE66AE66A3CDF7E
:1009C000E552E552E552E5521200380E816EB9DF6C
:1009D000320EE66EE66AE66AE66A2EDFE552E55218
:1009E000E552E552010E816EACDF320EE66EE66A2C
:1009F000E66AE66A21DFE552E552E552E5520D0E60
:100A0000816E9FDF320EE66EE66AE66AE66A14DF02
:100A1000E552E552E552E552060E816E92DF320E46
:100A2000E66EE66AE66AE66A07DFE552E552E552F7
:100A3000E5521200010E816E84DF0A0EE66EE66A50
:100A4000E66AE66AF9DEE552E552E552E552120041
:100A5000D9CFE6FFE1CFD9FF020E816E72DF0A0E19
:100A6000E66EE66AE66AE66AE7DEE552E552E552D8
:100A7000E552FD0EDBCFE6FFFE0EDB50280DF350F6
:100A8000E552E724E76EFE0EE7CFDBFFFD0EDB6AE3
:100A9000FE0EDB50F36EFD0EDBCFF4FFF350F45C83
:100AA00010E2140E816E4DDF010EE66EE66AE66A14
:100AB000E66AC2DEE552E552E552E552FD0EDB2A5A
:100AC000E7D7E552E7CFD9FF1200D9CFE6FFE1CF54
:100AD000D9FFFE0EDB50816E56DF010EE66EE66A30
:100AE000E66AE66AA9DEE552E552E552E552E552CC
:100AF000E7CFD9FF1200D9CFE6FFE1CFD9FFFD0E36
:100B0000DBCFE9FFFE0EDBCFEAFFEF500EE0FD0E7C
:100B1000DBCFE9FFDB2AFE0EDBCFEAFF01E3DB2AB6
:100B2000EF50E66ED2DFE552EAD7E552E7CFD9FFC4
:100B300012000201246B300E926EF00E936EEF0ED7
:100B4000206F20C281FF040E216F2151000825E291
:100B50002051FE0BE842206F20C281FF050EE66E99
:100B6000E66AE66AE66A68DEE552E552E552E55273
:100B70008150100B09E08150200B06E08150400BA2
:100B800003E08150800B01E10AD80201240502E153
:100B9000255104D02105216FD8D7CBD71200F00EF4
:100BA000936E81CF23F202012315226F0F0E2015C1
:100BB000206F20512211206F81CF23F2F00E2315D8
:100BC000226FF00E225D01E0F7D7936A06D826C2A5
:100BD00025F20201010E246F12000201276B100E94
:100BE000275D14E22751EA6A000FE96E020EEA223D
:100BF000EF50205D08E12751EA6A100FE96E020EFE
:100C0000EA22EFCF26F22729276FE9D726C281FFF4
:100C1000640EE66EE66AE66AE66A0EDEE552E552C4
:100C2000E552E55212000201286B070E285D1DE215
:100C300080DF0201296F2851EA6A2A0FE96E020E4D
:100C4000EA2229C2EFFF2851EA6A2A0FE96E020E52
:100C5000EA22EF50460802E108D004D029C2E6FF9C
:100C600034DFE5520201282BE0D72851EA6A2A0F27
:100C7000E96E020EEA22EF6A12000201286B070EEB
:100C8000285D16E22851EA6A2A0FE96E020EEA226E
:100C9000EF50E66E1ADFE55202012829EA6A2A0FB0
:100CA000E96E020EEA22EF5001E102D0282BE7D7CD
:100CB000120007DE80B80CD08128816EC80EE66E67
:100CC000E66AE66AE66AB8DDE552E552E552E552C3
:100CD00080BA0CD08104816EC80EE66EE66AE66AC0
:100CE000E66AAADDE552E552E552E55282B020D02F
:100CF000010E816E0201336B346B080E34AF02D0EB
:100D0000D89003D0335D000E345912E2C80EE66E5F
:100D1000E66AE66AE66A90DDE552E552E552E5529A
:100D20008150E824816E0201332B000E3423E5D775
:100D300082B218D081688080C80EE66EE66AE66AE4
:100D4000E66A7ADDE552E552E552E552816A809025
:100D5000C80EE66EE66AE66AE66A6EDDE552E552C0
:100D6000E552E5528250020B01E0010E026E825004
:100D7000010B016E8050200B01E0010E006E8050CF
:100D8000100B01E0010E00140114021420E0010E0A
:100D9000816E0201336B346B080E34AF02D0D890F1
:100DA00003D0335D000E345912E2640EE66EE66A3B
:100DB000E66AE66A41DDE552E552E552E5528150C8
:100DC000E824816E0201332B000E3423E5D772D75D
:020DD00012000F
:0E0DD2002A0EF66E080EF76E000EF86E020185
:100DE0000900F5503A6F0900F5503B6F03E13A678F
:100DF00001D03DD00900F550356F0900F550366F30
:100E00000900F550376F09000900F550E96E090037
:100E1000F550EA6E090009000900F550386F090025
:100E2000F550396F09000900F6CF3CF2F7CF3DF2DB
:100E3000F8CF3EF235C2F6FF36C2F7FF37C2F8FFF1
:100E40000201385302E1395307E00900F550EE6E14
:100E50003807F8E23907F9D73CC2F6FF3DC2F7FF81
:100E60003EC2F8FF02013A07000E3B5BBFD71200FB
:100E7000FF0EE350066E480E01D04C0EE76EE72ED3
:100E8000FED7E76AE72EFED7062EF7D7000012003E
:100E9000000EF36E00EE00F0080E01D81200EA60BA
:100EA00002D0EE6AFCD7F350E9601200EE6AFCD77C
:100EB00012EE40F022EE40F0F86A059CE9EC06F0F4
:0C0EC00066EC07F059EC06F0FBD71200BE
:020ECC00120012
:020ECE00EEED47
:100ED000EBE7DEDDDBD7BEBDBBB77E7D7B77303198
:0E0EE0003233343536373839414243444546C3
:00000001FF
